:020000040000FA
:0400000060283C3008
:08000800A000030EA100831209
:1000100005191028831601178312B2308100422877
:100020008316011383120B191C28AE17280A031913
:100030002E17AE192D283B28AE13AE192A282E1FD5
:100040003B28AE1A3B28A701A601A501A801AE01D5
:10005000AE164228F030AE0542282D152E13AE12F2
:100060002708AB002608AA002508A9002808AC002C
:10007000F030AE0542282E0DA80DA50DA60DA70D3A
:10008000AE1AAE0A8B100B11210E8300A00E200EAB
:02009000090065
:1000C000203084008001840A60300402031C62280E
:1000D000D6218316FF239000831283160C308505EA
:1000E000870183128501870107309900003083164C
:1000F00091009F008312C830831681008312313033
:100100009000003083168C00831210308B00472241
:1001100081018E018F010B118B100B108C130C13AE
:100120008C110C108B17AE202D19B020AA21B30B07
:10013000A128031085190314BA0DF0303A020319EF
:1001400021210C1C93280C10C00B93284108C000DF
:1001500085013F30831685008312932864000800D0
:10016000A91F2D11A91F0800291B2D11291B0800EB
:100170002B082A0629062C02031D2D11031D080039
:100180002D110130B7008B132030370783169B00E9
:100190001C141A088312A4001030370783169B0022
:1001A0001C141A088312A3000030370783169B0023
:1001B0001C141A088312A2008B1724082B02031D9B
:1001C0001B2923082A02031D1B2922082906F039AE
:1001D000A91EE039031D1B29220829050F3903191F
:1001E000032901303702031DFA283E18FA283E146D
:1001F000AD17F92102303702031D0329BE18032968
:10020000BE14AD170522290922050F3903191B2930
:1002100001303702031D11293E1C11293E10AD1774
:10022000112202303702031D1A29BE1C1A29BE10E2
:10023000AD171D221B29B70A033037020318080027
:10024000C328B601B301FA30B4000130B500013063
:10025000B70085018701AD1394213922AE20B30B7D
:100260005429031085190314BA0DF0303A0203190A
:100270008329B41F8501B41F8701B40B5429B50B22
:1002800054290230B5000130370203192F22023001
:100290003702031934223708B6080319B6000319C8
:1002A0005229B603FA30B4002D1D2E292D11A91F95
:1002B0002E29291B2E29A91E29120F3029050319C1
:1002C0002E29B9012918B90AA918B90A2919B90A90
:1002D000A919B90AB9182E2939192E298B132030DA
:1002E0003707BC002B08BB00B82110303707BC0013
:1002F0002A08BB00B82100303707BC002908BB0022
:10030000B8218B178E21402285018701B70AB601DB
:1003100003303702031C2E2947220800023037021F
:1003200003190800850187011430B900AE202D1D86
:1003300096292D11290A0319A129A91F9629291BDC
:1003400096290F302905031D9429B90B962985019B
:1003500087010800AD1F0800AD131030BC003E0837
:10036000BB00B8213030BC003F08BB00B8210800FA
:100370003C088B1383169B001C141A0883128B17DE
:100380003B02031908008B133B0883161C159A00C7
:100390003C089B0055309D00AA309D009C146400D1
:1003A0009C18CF291C1183128B170800831600306C
:1003B0009B001C141A088312BD00831610309B008A
:1003C0001C141A088312BE00831620309B001C14D4
:1003D0001A088312C1000130C11BC100C1080319F2
:1003E000C100831630309B001C141A088312BF0012
:1003F00008008316051085108312051085148E01E0
:100400008F010C104108C0000800831605128512E8
:100410008312051285168E018F010C104108C00051
:1004200008008316051085108312851005148E01AF
:100430008F010C104108C0000800831605128512B8
:100440008312851205168E018F010C104108C00021
:10045000080085013F3083168500831208003809A3
:1004600003398500B8000800380930398500B80024
:1004700008003C30831685008312B801B8140800C8
:100480000F30831685008312B801B81608000800E3
:084000000800000006000200A8
:02400E00CC01E3
:1042000001008100820084008800B100B200B40087
:10421000B800A100A200FF00FF00FF00FF00FF00A8
:104220000000010001000100010001000100010087
:10423000010001000100FF00FF00FF00FF00FF0080
:10424000010000000000000000000000000000006D
:10425000000000000000FF00FF00FF00FF00FF0063
:104260000000FF00FF00FF00FF00FF00FF00FF0055
:10427000FF00FF00FF00FF00FF00FF00FF00FF0046
:10428000FF00FF00FF00FF00FF00FF00FF00FF0036
:10429000FF00FF00FF00FF00FF00FF00FF00FF0026
:1042A000FF00FF00FF00FF00FF00FF00FF00FF0016
:1042B000FF00FF00FF00FF00FF00FF00FF00FF0006
:1042C000FF00FF00FF00FF00FF00FF00FF00FF00F6
:1042D000FF00FF00FF00FF00FF00FF00FF00FF00E6
:1042E000FF00FF00FF00FF00FF00FF00FF00FF00D6
:1042F000FF00FF00FF00FF00FF00FF00FF00DD00E8
:00000001FF
